:02000000942A40
:08000800532D82071034E83487
:1000100064340A3482072734033400340034303027
:10002000A600A700A800A900AA00B101B2013310E0
:1000300031080520B40031080A20B5003B20031820
:1000400036282630840031088407320880073108BA
:100050000520B40031080A20B500331043203108D0
:10006000033C03193828B10AB2011828B20A18282B
:100070002F08AA0708003310B409B5093408013E57
:10008000B4000318B50A3408AF0703183314350851
:10009000B007331C5128031850280130B0075128ED
:1000A000B00A08002E08AD06AE092C082B06AE05D6
:1000B000AD052E082D04AB05FF3A2C05AB04080056
:1000C0000630AF00AA20AF0B622886110611A420CB
:1000D0003830AF009320A020A4202830AF00932018
:1000E000A020A42028307B200F307B2001307B20F3
:1000F00006307B200800AF00861106119320A02057
:10010000AF0E9320A020A4202F0EFC390319AA20A3
:100110000800AF00861106159320A020AF0E932093
:10012000A020A420080006122F1A06168612AF1A65
:10013000861606132F1B06178613AF1B861708009B
:1001400086150000861108003430B0000000B00BA6
:10015000A62808001F30B100A420B10BAC2808006D
:1001600001307B2802307B28033904387B2807398B
:1001700008387B283F3940387B2880387B28061494
:100180000800AF000930B000031003180614031C68
:1001900006103230B1000000B10BCB28AF0CB00B11
:1001A000C52806143230B1000000B10BD428080075
:1001B0000830B200AF0DB00DB30D31083002331C62
:1001C0000318B0003318B30CB20BDA28AF0D0800D7
:1001D0009030B7003808BC00B81FF328B909B80937
:1001E000B90A0319B80AC1013808031DFD283908E6
:1001F000B80003193E29B901C1154108B702031D12
:10020000031C062A0310B81B0A29B90DB80DB70B39
:100210000329062ABC1FB81300343808BC00B817DD
:100220008030B702B71F03193E293708103CB700CA
:10023000031DB71B422908303702031C2729B700CA
:10024000B90D3808B900B801370803192C29031073
:10025000B80CB90CB70B27293D1B391C3629BA013C
:100260003A0DB9070319B80AB81B4229BC1F00345C
:10027000B909B809B90A0319B80A0034B801B901B3
:10028000B70100343D14BD1FFF34B801BC1FFF305F
:10029000B800B900BC0DB80CFF343708031D3E0888
:1002A00003193E2938083F06BC003E08B7078030D6
:1002B000031C5E29B707031893296129B707031C9C
:1002C000062AB817BF170310BA01BB011030C100CE
:1002D000391C70294008BB073F0803183F0FBA07B5
:1002E000BA0CBB0CB80CB90C0310C10B6829BA1BB3
:1002F0007D29B80DBB0DBA0DB7033D1B3B1C8C29E6
:10030000B80D0318BB0A0319BA0A031D8C29BA0CCD
:10031000BB0CB70A03189329BC1FBA133A08B800DC
:100320003B08B9000034BD14BD1FFF34FF30B700D7
:10033000B800B900BC0DB80CFF343E080319102AF0
:1003400038083F06BC00B817BF17C1013808BA000B
:100350003908BB004008BB023F08031C3F0FBA022C
:10036000BA01BB01031CBA290310B80CB90CBA0CB2
:100370000130C1003E08B702031CC4298030410788
:10038000B70703189329C92980304107B707031C11
:10039000062A1030C200BB0DBA0DB90DB80DC10D43
:1003A0004008B9023F08031C3F0FB8023F0DC104CB
:1003B000411CDC293B14E3294008B9073F08031816
:1003C0003F0AB8073B10C20BCB293D1B3B1CFF2942
:1003D0000310B90DB80DC10D4008B9023F08031C48
:1003E0003F0FB8023F0D41040139BB070318BA0A99
:1003F000031DFF29BA0CBB0CB70A03199329BC1FB4
:10040000BA133A08B8003B08B90000343D15BD1FC7
:10041000FF340130B700B801B901BC0DB80CFF348E
:10042000BD15FF348030BF0638083F06C1003708CD
:100430003E02031C2D2A3E08BA003708BE003A08C7
:10044000B7003F08BA003808BF003A08B8004008B3
:10045000BA003908C0003A08B9003808BC00B8171B
:10046000BF173F08BA004008BB003E083702BE0075
:1004700003194B2A08303E02031C432ABE00BB0D61
:100480003A08BB00BA013E0803194B2A0310BA0C04
:10049000BB0CBE0B462A3D1B3B1C5A2A031C5A2A86
:1004A000BB0A0319BA0A031D5A2ABA0CBB0CB70AB5
:1004B00003199329C11F612ABB09BA09BB0A031991
:1004C000BA0A3B08B9073A0803183A0FB807C11B24
:1004D000702A031C0A29B80CB90CB70F0A299329F2
:1004E0000318F328B909B809B90A0319B80A803002
:1004F000BC06F3283E08BA003708BE003A08B70029
:100500003F08BA003808BF003A08B8004008BA00EF
:100510003908C0003A08B90008003708BE0038089A
:10052000BF003908C000080083018B018A01203018
:1005300084008001840A7F300402031D992A9F01F0
:10054000850186018610831603133B308500003039
:10055000860005309F0081178312031341309F00EE
:100560000A30A1000530A200920191018B0183168F
:1005700003138C01831203138C0122309200831623
:100580000313F93092008C14831203130B178B178B
:100590001215A00160200430B720BF20A1253D170F
:1005A0000830F123A0188625201CD22A201005151A
:1005B0004825E63C031CE12A4C30F123201CDE2AAE
:1005C00020103330F123282420101930F123052482
:1005D00020102A30F1236B242010AB253B30F1236F
:1005E0002018F92AB22028257B24201DF52A201165
:1005F000F02A05118614B0202E25A001A301A40124
:10060000A501D4010530C8000030B8006430B9003D
:10061000E8208D220030B8000130B900E8209D218B
:100620003708D1003808D2003908D30028256C23B8
:10063000201C1E2B5D232010D80AB020A01C232BC9
:100640005D23A010AF23A01D182BA0115908031D76
:100650006623B220570A0739D700073A89200230AB
:10066000BD202825A624581CD8235818DF234A0863
:1006700047020318492BA01E182BA0121325B00106
:100680002408AF004808B100D820300803196C23B3
:10069000182B6C2386105C30F123E224D6255D23D1
:1006A00020182010A01C562BA010AF23A01D4F2BEC
:1006B000A0115908031D66234F2B2018622BA01888
:1006C000622B08000630D90066230800D90B6A2B7C
:1006D000051108000515080080305402031D9C2BED
:1006E00014304802031908002030AF00A030B000D9
:1006F000B100300884000008D50031088400550896
:100700008000B00AB00AB10AAF0B792B2030AF00DD
:100710002030B00030088400831700088313D50010
:100720003108840055088000B00AB00AB10AAF0B46
:100730008A2B0310C80DD40C541BA52B5408A03EC3
:1007400084004A088000D40A080054083F39203E3B
:1007500084004A08831780008313D40A08002017F6
:10076000E22420139C25D5015508AF00B0010F20CD
:100770002808C1202908C1202A08C1202C30C12006
:10078000551BC72B5508A03E84000008CE2B5508EA
:100790003F39203E840083170008831320177B24F1
:1007A00020139C25D50A55085402031DB42B0800BC
:1007B0004A087B24A624C724203089200800250865
:1007C000E9233A3089202408E92320308920E224D3
:1007D0000800AF00B0010F20290889202A088920CD
:1007E0000800D500B0205508831203178D0083162A
:1007F00003178C130C14831203178D0A0C08831231
:100800000313031908008920F72B0730BD200310BC
:10081000460C1E242E308920303046183530892071
:10082000201120180800AB1C112C201D112C2011A8
:10083000FA3046020319C601C60A052CAF00B00102
:100840000F2028088920290889202A0889200800E3
:100850003524201120180800AB1C2A2C201D2A2C1E
:10086000490A0339C9002011282C0A30BD203B2435
:10087000FF307B2408000030B800FF30B900E820CA
:100880008D2204308A004908033982074A2C502CF3
:10089000562C5C2C0930B800C430B900E820622C1A
:1008A0001330B8008830B900E820622C1D30B80041
:1008B0004C30B900E820622C3030B800D430B90098
:1008C000E820622C8A019D213708CB003808CC0033
:1008D0003908CD0008007624201120180800AB1C30
:1008E0006D2C201D6D2CC70A20116B2C0A30BD20E9
:1008F00047087B240800B900B801E8208D224B0886
:10090000B7004C08B8004D08B9004D210D21390839
:10091000AF003808B0000F20201B9B2C2608892030
:10092000270889202E308920280889202908892035
:100930005630892008002608C1202708C1202E3003
:10094000C1202808C1202908C12008004A08B90090
:10095000B801E8208D224B08B7004C08B8004D08BC
:10096000B9004D218D224608B900B801E8207A224D
:100970009D217A220030B8000230B900E8204D21D4
:100980003708CE003808CF003908D00008004E08DC
:10099000B7004F08B8005008B9000D213908AF0062
:1009A0003808B0000F202030892027088920280827
:1009B0008920290889202A0889206D308920413022
:1009C000892008000030B8003C30B900E8208D22B2
:1009D0005108B7005208B8005308B9009D210D21F5
:1009E0003908AF003808B0000F20201B082D26085A
:1009F00089202708892028088920290889202A0891
:100A000089206D3089204130892068308920080094
:100A10002608C1202708C1202808C1202908C12094
:100A20002A08C12008004E08B7004F08B800500837
:100A3000B9008D225108B7005208B8005308B90018
:100A400014223708D1003808D2003908D300080032
:100A50001F151F19292D1E08CA0008000301BA20FE
:100A60000830D6005603D50003193A2D00308920EE
:100A7000D50B362D5608083CD5000319432D1F30E1
:100A80008920D50B3F2D00308920D60B322D080050
:100A90009F15FF30AF00AF0B4B2D1F151F194E2DAB
:100AA0009F111E080800FE000308FF0083120313B5
:100AB0008C10A10B712D20150A30A100A20B712DF5
:100AC0000530A200A015A30A3C302302031D712D9E
:100AD000A016A301A40A3C302402031D712DA40119
:100AE000A50AAC01851E2C14051EAC145220451C11
:100AF0007B2D2B1C2014C51C7F2DAB1CA0142B0898
:100B0000C5007F088300FE0E7E0E0900A010B525EB
:100B1000D40803198E2D3B24AF2308004E30C1208A
:100B20006F30C1202030C1204430C1206130C1204D
:100B30007430C1206130C1200D30C1200A30C12085
:100B4000080046308400831203178D0183120313BB
:100B50000430F725080046308400831203178D0106
:100B600083120313043007260800513084008312D7
:100B700003177C308D00831203130430F725A03057
:100B800084008312031780308D00831203134030DA
:100B9000F72520308400831783120317C0308D009F
:100BA000831203134030F72583130800513084006B
:100BB000831203177C308D00831203130430072641
:100BC000A03084008312031780308D00831203133A
:100BD0004030072620308400831783120317C0306B
:100BE0008D00831203134030072683130800D500BD
:100BF000831603178C130C14831203170C08800040
:100C0000840A8D0A83120313D50BF82D0800D50032
:100C1000831603178C130C158312031700088C001E
:100C2000831603172126831203178D0A840A831261
:100C30000313D50B0C2E831603170C118312031309
:100C400008008B1355308D00AA308D008C148B1743
:060C50008C18282E08009C
:02400E00493F28
:084200006400990005000100B3
:104210004300610070002E0020004D006500740016
:104220006500720020005600200031002E0036008C
:1042300000004C006F00610064002000520020006C
:104240007800780078002E00780020006F00680069
:104250006D000000560020004300750074006F00E0
:1042600066006600000056002000520061006E00EB
:10427000670065000000780078002E007800780064
:10428000560020002000500072006500730073008B
:10429000200047004F0000002A002000420061007B
:1042A0007400740065007200790020006C006F00DB
:1042B000770020002A0000005200650061006400C1
:0A42C000790020002000200000001B
:0842F8000000000000000000BE
:00000001FF
